:012802005A7B
:03284800D22D226C
:03280B00022A3866
:03281300022AC9CD
:0428700090296A221F
:042878009029002281
:102900001053414D5000114341505455524500124F
:10291000434C530013434F50590014445241570045
:102920001544554D5000164C494E4500174D4F5615
:102930004500185155495400195254434745540015
:102940001A525443534554001B54454B001C4D45EB
:102950004153555245001D4556454E54001E494FA2
:10296000494E001F494F4F5554FF298A29CB2AF958
:102970002B062BA32BCA2C252C3E2B9E2C722C9F76
:102980002D7D2E5E2EAF2EDE2F08D293D290743F77
:10299000120030B40D01227439120030740112009B
:1029A000308980C290D2902091FDA2AFC2AF8547FE
:1029B0007085497185487292AF7580FFC293E5803A
:1029C000D293F87A0074A612003022D22ED212C20C
:1029D000AA743F120030B40D02805C7439120030CA
:1029E00074011200307440120030897B8B7C743982
:1029F000120030740112003089008B02BA0005B851
:102A000000028033857B82857C83E40AF0A3D8FCB6
:102A1000DAFA857B82857C83E9F0A3EBF0A374046A
:102A2000F57DF0A3E4F57EF0A3C212D2AAC22E5324
:102A300089F043A882D28C22C293C290D290D293C2
:102A4000C0E0C0F0C082C083E8C0E0E9C0E0857BA0
:102A500082857C83E0A3257BF8E0A3357CF9E0A3A5
:102A6000257BC0E0E0A3357CF583D0822091FDA2D8
:102A7000AFC2AF85477085497185487292AF758046
:102A8000FFC293E580D293F0A3E58288F0B5F017FA
:102A9000E58389F0B5F010857B82857C83A3A374E0
:102AA00004F0A3E4F08011857B82857C83A3A3E0FE
:102AB0002401F0A3E03400F0D0E0F9D0E0F8D083B6
:102AC000D082D0F0D0E0021BC7C0E0C082C083A299
:102AD000AFC2AF854774854975854876857B828509
:102AE0007C83A3A3E0A3F57DE0A3F57ED083D08211
:102AF000D0E092AFD216D0D032741FB1F2741BB1B5
:102B0000F2740CB1F22274391200307401120030E8
:102B1000C001C003744012003074391200307401D7
:102B2000120030C001C0037440120030743912002A
:102B30003074011200308B078906D002D000D00318
:102B4000D001EBB502004028E9B500004022BF00EB
:102B500005BE000280470F89828B83E0A3A982AB68
:102B60008388828A83F0A3A882AA83DEEADFE82230
:102B7000BF0005BE00028025E92EF9EB3FFBE82EE1
:102B8000F8EA3FFA0F19B9FF011B89828B83E0181D
:102B9000B8FF011A88828A83F0DEEADFE822741F18
:102BA000B1F22274391200307401120030C001C039
:102BB0000374401200307439120030740112003076
:102BC000E98BF0D083D082D1232274391200307483
:102BD00001120030C001C003744012003074391279
:102BE00000307401120030D002D00088828A83E065
:102BF000A328FEE0A33AFFE0A328FCE0A33AFDA847
:102C000082AA83BB0005B9000280198C828D830BD8
:102C1000E0B1F2A3EFB58308EEB5820488828A831F
:102C2000D9EEDBEC227439120030740112003074DA
:102C30001BB1F2E960011454072460B1F222743927
:102C40001200307401120030C001C0037440120041
:102C50003074391200307401120030B1FAE9F5799C
:102C60008BF085F07AD083858378D082858277D186
:102C7000232274391200307401120030C00191D542
:102C8000D0E06003F8E6F8E875F01084C0F075F065
:102C90000AA4D0F025F0F87A0074A612003022744D
:102CA000391200307401120030C00174401200303B
:102CB00074391200307401120030E975F00A84C0D2
:102CC000F075F010A4D0F025F0C0E091D5D0E0D0A0
:102CD00000F691F622B117B132F8B132F9B132FAF9
:102CE000B132543FFBB1325407FCB132FDB132FE78
:102CF000B132FFB12922B117E8B156E9B156EAB1B4
:102D000056EB543FB156EC5407B156EDB156EEB107
:102D100056EFB156B12922B12975F00474C5B156E8
:102D200064FFB156C4D5F0F62275F009B132D5F082
:102D3000FB22C082C083C0C643C604C0F09000041A
:102D400075F008C0E0E033D0E013D5F0F6D0F0D055
:102D5000C6D083D08222C082C083C0C643C604C00E
:102D6000F090000075F008C0E05401F582E0D0E07A
:102D700003D5F0F3D0F0D0C6D083D08222B1FA745C
:102D8000391200307401120030C001C003744012C7
:102D9000003074391200307401120030D002D000BB
:102DA00088828A83E0A328FEE0A33AFFE0A328FC00
:102DB000E0A33AFDA882AA83BB0005B900028031D6
:102DC0008C828D837C007D000BE0C082C0838C826E
:102DD0008D8375F000D107A3AC82AD83D083D08200
:102DE000A3EFB58308EEB5820488828A83D9DADB43
:102DF000D8223099FDC299F59922741FB1F2741B43
:102E0000B1F2741DB1F222C083C0822579C0E0E521
:102E1000F0357AF5F0E5822577F582E5833578F5AA
:102E200083D0E0C0E0C4035407A2F092E3A2F19281
:102E3000E44420B1F2D0E0541F4460B1F2E5835481
:102E400003C403F5F0E58203C4540745F04420B100
:102E5000F2E582541F4440B1F2D082D08322C29363
:102E6000C290D290D2932091FDA2AFC2AF8547709D
:102E700085497185487292AF7580FFC293E580D213
:102E800093F87A0074A6120030A871AA7274A61280
:102E90000030A8707A0074A612003078C87A0074E6
:102EA000A6120030740C120030740B12003022A8ED
:102EB0007DAA7E74A6120030A875AA7674A61200A8
:102EC00030A8747A0074A612003078C87A0074A60C
:102ED000120030740C120030740B12003022743F58
:102EE000120030B40D012274391200307401120046
:102EF0003089A07580FFC2B7E580D2B775A0FFF812
:102F00007A0074A612003022740112003089807495
:102F10003F120030B40D01227439120030740112D6
:0F2F2000003089A0C2B6D2B675A0FF7580FF221F
:00000001FF
